:100000009C0135298C007F3903198C000C208C1B36
:10001000FF3A8C1B013E08008A018207003403343A
:10002000063409340C3410341334163419341C34A7
:100030001F342234253428342B342E3431343334D5
:10004000363439343C343F34413444344734493411
:100050004C344E3451345334553458345A345C345F
:100060005E34603462346434663468346A346B34C9
:100070006D346F3470347134733474347534763451
:10008000783479347A347A347B347C347D347D34FA
:100090007E347E347E347F347F347F347F347F34CB
:1000A0007F347F347E347E347E347D347D347C34C2
:1000B0007B347A347A3479347834763475347434E1
:1000C0007334713470346F346D346B346A34683423
:1000D00066346434623460345E345C345A34583488
:1000E0005534533451344E344C3449344734443409
:1000F00041343F343C3439343634333431342E34A3
:100100002B342834253422341F341C34193416344B
:10011000133410340C3409340634033490001108BD
:100120009002031C910313089202031C930311080D
:100130008C0010080310900D910D900D910D9007FB
:100140000318910A0C08910713088C001208031079
:10015000920D930D920D930D92070318930A0C08BC
:1001600093072A210D309700980199019A019B016C
:100170009601200884001E08F12084136400C02822
:10018000100898070318990A1108990712089A0786
:1001900003189B0A13089B0719080220803E8D0054
:1001A0001B080220803E8D070D0C960700081E04D8
:1001B000031C1E068000170303190D309700031956
:1001C0008E0A03198F0FBE283029F5209E000408DF
:1001D000A0003029F5208004F128F520FF3A8005A1
:1001E000F228FF3A841780053029940006309419CC
:1001F0000530840001308A0014080739FF2882077F
:10020000013402340434083410342034403480344F
:100210008F018E006400FF308E07031C8F07031CC4
:10022000080003308D00DC3017210A298D01E83EDB
:100230008C008D09031C2129FC308C0703181D2913
:100240008C078D0F1C298C1825298C1827290C1830
:10025000292908008E098F098E0A03198F0A0800C0
:1002600083130313831264000800932185217621F0
:10027000762101308F002C300921762185218521BE
:1002800001308F002C300921852185218521852190
:10029000762101308F002C3009217621852185219E
:1002A000852101308F002C300921852185210130E5
:1002B0008F002C30092185218521852101308F0077
:1002C0002C300921A1210130E52060308E00EA3078
:1002D0008F00033093009100E83092008E20CE21F1
:1002E0009C21EA308F006030092135290130E5205A
:1002F0002C308E0001308F00043093009100B0301C
:1003000092008E206430082108000130E52064301E
:100310008E008F01043093009100B03092008E2047
:100320006430082108000030EA200330ED2001305D
:100330008F002C30092108000030ED200330EA2026
:1003400008000130E52064308E008F0101309300F9
:100350009100F43092008E200130E52064308E0050
:100360008F01023093009100583092008E200130AE
:10037000E52064308E008F01023093009100BC3084
:1003800092008E200130E52064308E008F01033012
:1003900093009100203092008E2008000130E5206B
:1003A00064308E008F010330930091002030920062
:1003B0008E200130E52064308E008F0102309300E2
:1003C0009100BC3092008E200130E52064308E0018
:1003D0008F01023093009100583092008E2001303E
:1003E000E52064308E008F01013093009100F430DD
:0603F00092008E200800BF
:084000007F007F007F007F00BC
:04400E00F53F010079
:00000001FF
